:10033400453100453000011A3F80000001123F8022
:10034400000004123E80000008123E0000000C125F
:100354003DAAAAAB18123D2AAAAB32123CA3D70A73
:06036400C8123BA3D70AFA
:10003C007526007527007528A4752905E4F52AF5A1
:0E004C002B752C00752DA1752E031224112288
:10005A0078AEE678A4F678AFE678A5F678B0E678D2
:10006A00A6F678B1E678A7F678B2E678A8F6782008
:10007A00E2FC08E2FD08E2FE08E2FF7829122BA55D
:10008A007824E2FC08E2FD08E2FE08E2FF782F127B
:03009A002BA52271
:0B009D00300905C288D2A822D2AC2294
:0E00A800E4FF7F207800E4F208DFFC751A0008
:0100B6002227
:1000B700300875785F7401F2E408F2784F122BB1BB
:1000C700412000007853122BB141200000783312F1
:1000D7002BB141C80000784774FDF20874E8F2E4D8
:1000E70008F208F20874FDF20874E8F2E408F2086E
:1000F700F27857122BB13F800000785B122BB13F8B
:100107008000007837122BB13F800000783F122B18
:10011700B100000000783B122BB13F80000078430C
:0E012700122BB100000000221210A780FB2254
:10013500122324120BE5300E0C1210A71210A71271
:0901450010A71200B71210A72246
:10014E00C2AF78AD760118760118760118760118CF
:10015E007601E418F618F618F618F618F612003CA2
:10016E001211163009051211B4800312134EE4F564
:10017E0018C203C20DC20CC206C20BC20FC205C208
:10018E0001C20AC202C207C2001200A812013578CB
:10019E004FE2FB08E2F908E2FA08E2CBF87F007EB4
:1001AE00007D807C3F1226B27890122B997853E214
:1001BE00FB08E2F908E2FA08E2CBF87F007E007D48
:1001CE00807C3F1226B2788C122B99E4F515AF1570
:1001DE00121039AF15121067120F4D120F88120F31
:1001EE00C3120FFE12037112005A12003C120F17A7
:0601FE0012009DD2AF22A9
:08020400E517700312005A22F5
:10020C00E51024D0B40800503E90021CF828287346
:10021C0002023402023802023C0202400202440290
:10022C00024802024C020250121BE322121BE32270
:10023C00121A0A2212198C221219CB22121AAB2270
:08024C0012225A22121F99220E
:10025400200112E51064306005E510B43105AF16D5
:06026400120D1DC20F2265
:10026A00C2AF1211AA12013512003C120D1778A35F
:08027A00E630E2F412014E220D
:10028200300B361207A21200A830070512113CC229
:1002920007C20B12020420052030041D2003033084
:1002A2000D0B7BFF7A03793412194A80097BFF7A9E
:1002B20003793712194A12198312003C120D793050
:1002C200050312020C300F0312025478A3E620E257
:0B02D2000312026A121104120D172221
:1002DD00300B101207A2C20B1200A81211F5120258
:1002ED0004D2AF12003C120D79300506200B03121B
:1002FD00020C300F06200B0312025478A3E620E205
:10030D000312026A12121130070512120AC20712E5
:06031D0010D0120D1722A2
:1003230012014E3009051202DD80FB12028280FBAE
:0103330022A7
:1007F300256600253163003A010000000000000077
:1008030000000000000000FF036BFF15F33B000234
:1008130000000000000000000000000000FF036B68
:10082300FF036A3C0000000000000000000000001D
:10083300000000FF036BFF036A3D0100000000009E
:10084300000000000000000000FF036BFF18C03E23
:100853000202000000003F7AE1483F828F5C00FF04
:10086300036BFF185C3F0100000000000000000064
:100873000000000000FF036BFF15E94002020000C7
:1008830000003F7AE1483F828F5C00FF036BFF1853
:100893006741020200000000000000007E96769986
:1008A30000FF036BFF17EF4202010000000000008E
:1008B30000003F80000000FF036BFF155C43020351
:1008C3000000000000000000477FFF0000FF036BF3
:1008D300FF183A44020400000000C700000046FF6E
:1008E300FE0000FF036BFF184B45000100000000F2
:1008F300000000000000000000FF036BFF036A46D6
:10090300010100000000000000003F80000001FF23
:10091300036BFF15444701010000000000000000C5
:100923003F80000001FF036BFF1524480000000017
:100933000000000000000000000000FF036BFF0345
:100943006A49010200000000FE9676997E96769928
:1009530001FF161CFF16B44A02030000000000004A
:100963000000477FFF0000FF036BFF18184B0204D2
:1009730000000000C700000046FFFE0000FF036BFD
:10098300FF18294C000000000000000000000000D8
:10099300000000FF036BFF036A4D0101000000002C
:1009A3000000000040E0000001FF036BFF14264E2F
:1009B3000101000000000000000040E0000001FF12
:1009C300036BFF14D34F020200000000BE4CCCCDDA
:1009D3003E4CCCCD00FF036BFF1889500101000092
:1009E3000000000000003F80000001FF036BFF15C3
:1009F3002C510202000000003F8000003FB333335C
:100A030000FF036BFF187252010300000000000097
:100A130000004150000001FF036BFF156553010106
:100A230040A000000000000040E0000001FF036B55
:100A3300FF143954000100000000000000003F8053
:100A4300000001FF036BFF036A5501020000000071
:100A5300FE9676997E96769901FF15FDFF173D5612
:100A6300020200000000000000007E96769900FF5D
:100A7300036BFF17C65702000000000000000000D0
:100A83000000000000FF036BFF0C6A580100000028
:100A93000000000000000000000001FF036BFF15D1
:100AA3001859010100000000000000004000000090
:100AB30001FF036BFF14155A02050000000000003C
:0D0AC30000000000000000FF036BFF18A002
:01036A002270
:02036B00C322AB
:04036D00122C252207
:10037100E478A0F678A0E6F9C3942140030204458D
:1003810075F016E9A42409F582E5F03408F583E453
:10039100936401600302043F75F016E9A424FCF59F
:1003A10082E5F03407F583E493FBB4021775F01688
:1003B100E9A424FDF582E5F03407F583122B6C786E
:1003C100B8122B99EBB4012475F016E9A424FDF5BC
:1003D10082E5F03407F583122B6C7B007A007940BB
:1003E10078421224B812280778B7A60778A0E6FF4A
:1003F10075F016A424FCF582E5F03407F583E49347
:10040100B4031C75F016EFA424FDF582E5F0340762
:10041100F583122B6C1228077882A60608A60778A6
:10042100A0E675F016A4240DF582E5F03408F583F5
:10043100E493FB740193FA740293F912036D78A0AB
:0904410006020375C203C20D227C
:10044A00C211781F740AF278A0E675F016A424FC8B
:10045A00F582E5F03407F583E49314700302057717
:10046A0024FE70030204F61470030205F3147003E9
:10047A0002067124036003020689A91A7A007BFE28
:10048A00C0030B8B28752907752AF3752B00752C69
:10049A0000752DB8D0031231DF8F24E52464017072
:1004AA004678A0E675F016A42401F582E5F0340832
:1004BA00F583122B6C78B8122B7C12274B402378C9
:1004CA00A0E675F016A42405F582E5F03408F58354
:1004DA00122B6C78B8122B7C12274B600250030245
:1004EA000689D211020689D211020689A91A7A004E
:1004FA007BFEC0030B8B28752907752AF3752B0021
:10050A00752C00752DB8D0031231DF8F24E52464D1
:10051A0001705578A0E675F016A42401F582E5F07D
:10052A003408F583122B6C78B8122B7C12274B40B7
:10053A002078A0E675F016A42405F582E5F03408C3
:10054A00F583122B6C78B8122B7C12274B6007406C
:10055A0005D21102068978B8122B60122807788210
:10056A00A60608A607020689D211020689A91A7ADE
:10057A00007BFEC0030B8B28752907752AF6752B9D
:10058A0000752C00752DB7D0031231DF8F2478B790
:10059A00E6FF12369B4002D21178B7E624D0FCE47B
:1005AA001227D378A0E675F016A42401F582E5F0A7
:1005BA003408F583122B8912274B6002502678B72C
:1005CA00E624D0FCE41227D378A0E675F016A4241A
:1005DA0005F582E5F03408F583122B8912274B4082
:1005EA0003020689D211020689A91A7A007BFEC083
:1005FA00030B8B28752907752AF3752B00752C00B8
:10060A00752DB8D0031231DF8F24E52464017053AD
:10061A0078A0E675F016A42401F582E5F03408F511
:10062A0083122B6C78B8122B7C12274B402078A0AF
:10063A00E675F016A42405F582E5F03408F5831270
:10064A002B6C78B8122B7C12274B60064004D2110F
:10065A00802D78B8122B601228077880A60608A683
:10066A0007801CD2118018C3741F951AFF74009456
:10067A0000FED3EF940CEE648094804002D21120E5
:10068A00112078A0E675F016A4240AF582E5F03464
:10069A0008F583E493740193FA740293F9122C25F2
:0406AA009211A211F6
:0106AE002229
:1006AF00C211A81AE2FF7004D2118031EF24C6786C
:1006BF00A0F675F016A424FBF582E5F03407F58358
:1006CF00E49314600B14600C24027011D211800D8E
:1006DF00C2118009300804C2118002D211051AA27A
:0106EF0011F9
:0106F00022E7
:1006F100E4F52474002524F8E2FFC3648094E1400A
:1007010012D3EF648094FA500A1236C07400252483
:10071100F8EFF274002524F8E2FFC3648094AD4041
:1007210008D3EF648094DA4022EF642F601DAF2478
:10073100D3EF64809481400F74FF2FF8E2FE7400C0
:100741002FF8EEF21F80E9E47800F20524C3E524D6
:060751006480949F409DAE
:01075700227F
:10075800C3741F951AFEEE601B781FE2FF7D1F749D
:10076800FF2DF8E2FC74002DF8ECF2DDF27800EFD2
:04077800F21E80E20B
:01077C00225A
:10077D00751A1FE51AD39400401A151AA81AE2FF2C
:10078D00C3648094BA40ECD3EF648094DA50E4EF04
:05079D00644560DF224D
:1007A2001207581206F112077D1206AF92033003A8
:1007B20002D20C20030A12044A920D300D02D20614
:1007C200200322200D1F78A0E675F016A4240DF553
:1007D20082E5F03408F583E493FB740193FA740222
:1007E20093F912036D300303D20C22300D02D206AC
:0107F20022E4
:090AD000752DA08F2E1223B72210
:100AD9008B268A2789288D29D3E52964809481402A
:100AE90022752DA01223E1AB26AA27A928EF122AE5
:100AF90091152974012528F528E43527F527120DC4
:100B09001780D5752DA01223FBAB26AA27A928EF9C
:040B1900122A9122E9
:100B1D008B268A2789288D29D3E5296480948040E6
:100B2D0022752DA01223E1AB26AA27A928EF122AA0
:100B3D0091152974012528F528E43527F527120D7F
:040B4D001780D52216
:080B51008B278A2889298D2ACF
:100B5900D3E52A64809480402AAB27AA28A92912C0
:100B69002A29F52C752DA0852B2EF52F12239715E3
:100B79002A74012529F529E43528F528052B120DB4
:050B89001780CDAF2B29
:010B8E002244
:080B8F008B288A29892A8D2B8D
:100B9700E4F52FC3E52B6480F8E52F648098502493
:100BA700AB28AA29A92A122A29AB2CAA2DA92E12C9
:100BB7002A6F7401252AF52AE43529F529120D171C
:040BC700052F80CFA7
:010BCB002207
:100BCC00E4F5277D3AF52C752D00752E277BFE7AE2
:080BDC00007933120B8FAF27E3
:010BE40022EE
:100BE500C20EE4FF120AD07B007A0079247D01123F
:100BF5000B1DE52464A06002D20E7B007A007924E7
:100C05007D01120B1DE524647C6002D20E7B007A07
:100C15000079257D01120B1D7B007A0079247D0169
:100C2500120B1D7B007A0079247D01120B1D7B00C0
:100C35007A0079247D01120B1D7B007A0079247DD1
:100C450001120B1D7B007A0079247D01120B1D7B9F
:100C5500FE7A0079337D3A120AD9120BCCEF65255D
:040C65006002D20E49
:010C69002268
:100C6A00E4F5267525A0FB7A0079257D0185262BDA
:100C7A00120B518F2675257C7B007A0079257D0120
:100C8A0085262B120B518F26120BCC8F257B007ACF
:100C9A000079257D0185262B120B518F267525FF9C
:100CAA007B007A0079257D0185262B120B518F2630
:100CBA007525FF7B007A0079257D0185262B120B8D
:100CCA00518F267525FF7B007A0079257D018526BF
:100CDA002B120B518F267525FF7B007A0079257D13
:100CEA000185262B120B518F267525FF7B007A0072
:100CFA0079257D0185262B120B518F267BFE7A00E2
:0C0D0A0079337D3A85262B120B518F2681
:010D160022BA
:060D1700904000E4F02210
:100D1D008F24120F17D20178A97601087601087673
:100D2D0001087611087620AF16EF3395E0FE90039B
:100D3D003B75F006EF122BCAEE75F006A42583F570
:100D4D0083E4934420F612003C78A97601087601DD
:100D5D0008760108760108760178287401F2786F1B
:0C0D6D00122BB100000000E4782DF222EF
:100D7900200103020F1678A3E630E103020ED2AF79
:100D890016EF3395E0FE90033A75F006EF122BCA81
:100D9900EE75F006A42583F583E493FD7828E26DCA
:100DA9006003020E8278A9760108760108760108A7
:100DB900761108762190033B75F006EF122BCAEEE7
:100DC90075F006A42583F583E4934421F612003CCB
:100DD90078AD760118760108763912003C78AD763F
:100DE9000178A1E6F52508E6F524786FE2FB08E22B
:100DF900F908E2FA08E2CBF8AE24AF25E4FCFDEBF2
:100E09002FFFEA3EFEED39FDEC38FC786F122BA579
:100E1900786FE2FC08E2FD08E2FE08E2FFE412272F
:100E2900C9AB16EB3395E0FA90033C75F006EB126B
:100E39002BCAEA75F006A42583F583122B8912259E
:100E4900A97B007A00798078371225A98F148E132F
:100E59008D128C1178B3122B7C1224B48F148E133B
:100E69008D128C11789C122B7C1225A98F148E134C
:100E79008D128C11D20AC2012278A9760108760155
:100E890008760108760108763912003C78AD7601BA
:100E990078A1E6F52508E6F524786FE2FB08E2F982
:100EA90008E2FA08E2CBF8AE24AF25E4FCFDEB2F0B
:100EB900FFEA3EFEED39FDEC38FC786F122BA57880
:100EC90028E204F2E4782DF222782DE2C3945A50F4
:100ED90004E204F22275140075130075128075116D
:100EE9003FAF14AE13AD12AC1178B3122B7C1224A0
:100EF900B48F148E138D128C11789C122B7C1225B1
:0D0F0900A98F148E138D128C11D20AC20113
:010F160022B8
:100F170078AD76FF1876FF1876FF1876FF1876FFFC
:100F270012003C78A97621E408F608762108F6082D
:100F3700760112003C78A976010876010876010847
:060F47007601087601228C
:100F4D007847E2FC08E2FDE41227CE7888122B994F
:100F5D007888122B607B007A00798078471224B84C
:100F6D007888122B997888122B607B007A00790093
:0B0F7D00783F1225A97888122B9922DA
:100F88007849E2FC08E2FDEC1227CE7898122B99FA
:100F98007898122B607B007A007900783F1224B889
:100FA8007898122B997898122B607B007A00790038
:0B0FB800783F1225A97898122B99228F
:100FC300784BE2FC08E2FDE41227CE7884122B99D9
:100FD3007884122B607B007A00798078471224B8DA
:100FE3007884122B997884122B607B007A00790025
:0B0FF300783F1225A97884122B992268
:100FFE00784DE2FC08E2FDEC1227CE7894122B9984
:10100E007894122B607B007A007900783F1224B816
:10101E007894122B997894122B607B007A007900C9
:0B102E00783F1225A97894122B99221C
:10103900EF25E025E02437F8E2FC08E2FD08E2FEAE
:1010490008E2FF789C122B99789C122B607B007A1E
:0E10590000790078401225A9789C122B99226C
:10106700EF25E025E0243FF8E2FC08E2FD08E2FE78
:1010770008E2FF78B3122B9978B3122B607B007AC2
:0E108700007900783F1224B878B3122B99221A
:09109500D295D297D296D2942292
:09109E00C295C297C296C29422C9
:1010A70012109EE4FFFE120D170FBF00010EBE3E89
:1010B700F5BF80F2121095E4FEFF120D170FBF0067
:0810C700010EBE3EF5BF80F2F0
:0110CF0022FE
:1010D000908004E030E104C2968002D296908002B3
:1010E000E030E404C2948002D294908004E030E2C4
:1010F00004C2978002D297908003E030E603C29545
:0411000022D2952240
:10110400300B04C2978002D297300203C29622D2D7
:02111400962221
:1011160090C000E020E704D2088002C20890C00018
:10112600E030E603D20922C20990C000E030E403B1
:06113600D20422C20422D3
:10113C00120135E478A8F6784FE2FB08E2F908E2F0
:10114C00FA08E2CBF87F007E007D807C3F1226B24D
:10115C007890122B997853E2FB08E2F908E2FA082E
:10116C00E2CBF87F007E007D807C3F1226B2788C2B
:10117C00122B99120F17C201E4F515AF1512103985
:10118C00AF15121067120F4D120F88120FC3120FEA
:0B119C00FE12037112005A12003C22E8
:0311A700C2A822B9
:0A11AA001211A79080057402F022D4
:1011B4009080057402F0908001740BF0A37401F028
:1011C4009080057422F07486F074A8F09080047402
:1011D40001F090800674E0F090C000E0541F90800D
:1011E40006F090800574C1F0E4F0908007740AF072
:0111F40022D8
:0711F5009080057403F02255
:0711FC00908005740FF02242
:071203009080057406F02243
:07120A0012113C1211FC223D
:10121100908003E020E636E4FF78A3E6FE5480FDEB
:101221003395E04D60027F02EE30E6034307047818
:101231006DE26F5FFE786EE25E6009EF4440908080
:0D12410003F08005908003EFF0786DEFF270
:01124E00227D
:10124F00751A00D202E51A04F8E27007121203C2EF
:10125F0002D200A81AE2908000F0E51AC3941F5042
:10126F0002051A300012E4FF7F1F7800E4F208DF56
:08127F00FC7F1F751A00C2007C
:011287002244
:030003000212885E
:0B128800C0E0C083C082C0D075D00859
:10129300908001E0FFA3E030E002C202EF30E01FE4
:1012A300C205908000E0A81AF2E51AC3941F500407
:1012B300051A8003751A00EF30E404D20BC2AFEFB6
:1012C30030E14020020AD205E5187037D20F80338F
:1012D300E51A04F8E27007121203C202D200A81A38
:1012E300E2908000F0E51AC3941F5002051A300003
:1012F30012E4FE7E1F7800E4F208DEFC7E1F751AFE
:0913030000C200EF30E302D20742
:09130C00D0D0D082D083D0E032B1
:10131500E4FCFD7B20FAF9F8122AC2A804A905AA63
:1013250006AB077F007E1B7DB77C0012361AC3E42F
:101335009FF525E49EF524759852E4F5C875C830E7
:081345008525CA8524CBD2CA1C
:01134D00227D
:10134E0090C000E0540314601214601714601C2443
:10135E0003701F7FB07E04121315227F607E091268
:10136E001315227FC07E12121315227F807E251246
:03137E0013152222
:10138100751A00C299A81AE2600BD202051AE51A71
:0613910014F8E2F59922B8
:030023000213972E
:07139700C0E0C0D075D008D2
:10139E00309948C299300243A81AE2FF6026F599A7
:1013AE00E51AC3941F5004051A8030751A00E51A09
:1013BE00D3941F5008A81AE4F2051A80F1751A008A
:1013CE00C2028017751A00E51AD3941F5008A81A86
:1013DE00E4F2051A80F1751A00C202309824AF9912
:1013EE00200B1D20021A200517A81AEFF2E51AC3CA
:1013FE00941F5004051A8003751A00BF0D02D20BFC
:02140E00C29882
:05141000D0D0D0E03255
:0318C3002573008A
:1014150030090878B7E624D0F51922D203E4F51986
:0114250022A4
:1014260030090978B7E624D0796EF322D203E4783E
:031436006EF22231
:1014390078B7E624D0F516120F1778A97601087641
:1014490001087601087611087660AF16EF3395E04A
:10145900FE90033B75F006EF122BCAEE75F006A459
:101469002583F583E4934460F612003C78AC760159
:10147900087601E4782DF212003C782DE204F27826
:10148900A3E630E108782DE2C394B440EA78AC765B
:1014990011087621AF16EF3395E0FE90033B75F006
:1014A90006EF122BCAEE75F006A42583F583E493A3
:1014B9004421F612003C78AD760118760108763998
:0A14C90012003C78AD7601C201224A
:1014D30078B7E6F510E51024CF601C04703278B2BB
:1014E300E64401F6E5156028E4F515AF151210671B
:1014F300AF15121039801978B2E654FEF6E515647B
:1015030001600D751501AF15121067AF1512103973
:05151300E4782EF22235
:0C151800E517B4010612005A12003C2234
:0815240078B7E624D0F5172288
:10152C0078B7E624CF600A04700D78B2E6547FF6E3
:08153C002278B2E64480F62299
:1015440078B7E624CF600A04700D78B2E654BFF68B
:081554002278B2E64440F622C1
:09155C0078B7E624D0795FF32290
:101565007882E6FC08E6FDD39407EC9400502A7EC9
:1015750000ED5407FF18EEF608EFF67803C333CEF7
:1015850033CED8F97983F7EE19F778B2E654C7FF69
:10159500F67883E64F78B2F622EC703EED24F760DC
:1015A5001714601B14601F14602314602724057032
:1015B5002978B2E654F7F62278B2E64408F622789E
:1015C500B2E654EFF62278B2E64410F62278B2E697
:0B15D50054DFF62278B2E64420F62234
:0915E000D205E5187002D20F22B9
:0A15E9002009041215E022D20322AB
:0A15F300200904121BF522D2032286
:1015FD0078B8122B60123472784FE2FB08E2F908CA
:0F160D00E2FA08E2CBF812274B5002D322C32295
:10161C0078B8122B601234727853E2FB08E2F908A6
:0F162C00E2FA08E2CBF812274B5002D322C32276
:10163B008F2C8E2B8D2A8C29AB30AA2FA92EA82D5F
:10164B001225A98F2C8E2B8D2A8C29AB34AA33A96A
:10165B0032A8311224B88F2C8E2B8D2A8C2912286C
:10166B00077BFF7AFF79007800C3122B1F50097F8D
:10167B00FF7EFF7D007C0022AF2CAE2BAD2AAC2968
:10168B001228077B017A0079FF78FFD3122B1F40BA
:10169B00097F017E007DFF7CFF22AF2CAE2BAD2A94
:0916AB00AC2912347F1228072239
:1016B400788C122B6078B8122B7C1225A978201212
:1016C4002BA57884122B608F308E2F8D2E8C2D7845
:1016D40094122B608F348E338D328C317820E2FC5F
:1016E40008E2FD08E2FE08E2FF12163B8F288E276F
:1016F4008D268C25E526603378B2E64404F6AF28BF
:10170400AE27AD26AC25EC1227C9785BE2FB08E2D4
:10171400F908E2FA08E2CBF81225A91227B8122830
:10172400078F288E278D268C25800678B2E654FBF9
:08173400F678AFA62818A627DD
:01173C00228A
:10173D007890122B6078B8122B7C1225A978241280
:10174D002BA57888122B608F308E2F8D2E8C2D78B7
:10175D0098122B608F348E338D328C317824E2FCCD
:10176D0008E2FD08E2FE08E2FF12163B8F288E27E5
:10177D008D268C25E526603378B2E64402F6AF2837
:10178D00AE27AD26AC25EC1227C97857E2FB08E24F
:10179D00F908E2FA08E2CBF81225A91227B81228A7
:1017AD00078F288E278D268C25800678B2E654FD6E
:0817BD00F678B1A62818A62752
:0117C5002201
:1017C60078B8122B60784F122BA5784FE2FB08E20F
:1017D600F908E2FA08E2CBF87F007E007D807C3FC4
:0917E6001226B27890122B992210
:1017EF0078B8122B607853122BA57853E2FB08E2DE
:1017FF00F908E2FA08E2CBF87F007E007D807C3F9B
:09180F001226B2788C122B9922EA
:101818007882E6FF08E67847CFF208EFF2120F4D1C
:01182800229D
:101829007880E6FF08E67849CFF208EFF2120F88D0
:01183900228C
:10183A007882E6FF08E6784BCFF208EFF2120FC380
:01184A00227B
:10184B007880E6FF08E6784DCFF208EFF2120FFE34
:01185B00226A
:0B185C0078B8122B607857122BA522E1
:0B18670078B8122B60785B122BA522D2
:1018720078B8122B60E51525E025E02437F8122B05
:07188200A5AF151210392279
:1018890078B8122B60E51525E025E0243FF8122BE6
:07189900A5AF151210672234
:1018A000A91A7A007BFEC0030B8B28752918752AAC
:1018B000C31B8B2B752C00752D60D0031231DF22DA
:0318C000D207222A
:10228E002573000D0A00000D00000A0D0000252B1D
:10229E002E354500494234302056312E333000253C
:1022AE002B2E3545564F00252B2E3545564E0025E7
:1022BE002B2E3545414F00252B2E3545414E002501
:1022CE006300252B2E35454100252B2E354542002A
:1022DE00252B2E35454300252B2E35454400252B29
:1022EE002E35454500252B2E35454600252B2E3502
:1022FE00454700252B2E35454800252B2E354549C3
:10230E0000252B2E35454A00252B2E35454B002515
:06231E002B2E35454C009A
:0D18C60030090412124F22D2AF12138122FA
:1018D300E51914604E04706E300924A91A7A007B4E
:1018E300FEC0030B8B2C752D22752E8E8B2F75301E
:1018F30022753191D003122D61EF251AF51A22A911
:101903001A7A007BFEC0030B8B2C752D22752E8E4D
:101913008B2F753022753195D003122D61EF251A67
:10192300F51A22A91A7A007BFEC0030B8B2C752DA6
:1019330022752E8E8B2F753022753198D003122D80
:0719430061EF251AF51A22DD
:10194A008B248A258926C2AF751A00AB24AA25A939
:10195A0026122A29FF6019A81AF274012526F526EB
:10196A00E43525F525E51AC3941F50DF051A80DBF7
:09197A001218D31218C6D2AF22D4
:09198300300205120D1780F82254
:10198C00C2AF751A00A91A7A007BFEC0030B8B2C10
:10199C00752D22752E9C784FE2FC08E2FD08E2FEC4
:1019AC0008E2F5328E318D308C2FD003122D61EF81
:0F19BC00251AF51A1218D31218C6C205D2AF2277
:1019CB00C2AF751A00A91A7A007BFEC0030B8B2CD1
:1019DB00752D22752E9C7853E2FC08E2FD08E2FE81
:1019EB0008E2F5328E318D308C2FD003122D61EF42
:0F19FB00251AF51A1218D31218C6C205D2AF2238
:101A0A00C2AF78A3E6FF30E70778007431F28005A9
:101A1A0078007430F2EF30E60778017431F280050D
:101A2A0078017430F2785FE27012EF30E5077802DD
:101A3A007431F2801978027430F2801278A8E63094
:101A4A00E60778027431F2800578027430F2EF30DA
:101A5A00E40778037431F2800578037430F2EF30CA
:101A6A00E30778047431F2800578047430F2E4FFF5
:101A7A003008010F300E027F02EF24307805F27F22
:101A8A00303006027F32300C027F317806EFF2C224
:101A9A0006C20C751A071218D31218C6C205D2AF9D
:011AAA002219
:101AAB00C2AF7BFF7A2279A212194AC205D2AF22AA
:101ABB00751A00E51024CF7003021B580460030253
:101ACB001BDFAF14AE13AD12AC11784FE2FB08E283
:101ADB00F908E2FA08E2CBF81225A98F148E138DC0
:101AEB00128C11123472784FE2FB08E2F908E2FA19
:101AFB0008E2CBF812274B502AA91A7A007BFEC0BA
:101B0B00030B8B2C752D22752EAD8514328513315D
:101B1B0085123085112FD003122D61EF251AF51A7E
:101B2B00021BDFA91A7A007BFEC0030B8B2C752DD1
:101B3B0022752EB585143285133185123085112F00
:101B4B00D003122D61EF251AF51A021BDFAF14AE6D
:101B5B0013AD12AC117853E2FB08E2F908E2FA0874
:101B6B00E2CBF81225A98F148E138D128C1112341F
:101B7B00727853E2FB08E2F908E2FA08E2CBF812BA
:101B8B00274B5029A91A7A007BFEC0030B8B2C75AF
:101B9B002D22752EBD85143285133185123085119A
:101BAB002FD003122D61EF251AF51A8027A91A7A67
:101BBB00007BFEC0030B8B2C752D22752EC5851457
:101BCB003285133185123085112FD003122D61EF21
:081BDB00251AF51A1218D32295
:101BE300300A0EC2AF121ABB1218C6C20AC205D2FD
:021BF300AF221F
:101BF500751A00A91A7A007BFEC0030B8B2C752D74
:101C050022752E9C784FE2FC08E2FD08E2FE08E210
:101C1500F5328E318D308C2FD003122D61EF251AC0
:101C2500F51A1218D31218C6121983751A00A91AB3
:101C35007A007BFEC0030B8B2C752D22752E9C78AC
:101C450053E2FC08E2FD08E2FE08E2F5328E318D32
:101C5500308C2FD003122D61EF251AF51A1218D3E7
:101C65001218C6121983751A00A91A7A007BFEC0CC
:101C7500030B8B2C752D22752E9C7837E2FC08E220
:101C8500FD08E2FE08E2F5328E318D308C2FD0034F
:101C9500122D61EF251AF51A1218D31218C612194A
:101CA50083751A00A91A7A007BFEC0030B8B2C756D
:101CB5002D22752E9C783FE2FC08E2FD08E2FE0825
:101CC500E2F5328E318D308C2FD003122D61EF2548
:101CD5001AF51A1218D31218C6121983751A007834
:101CE50047E2FC08E2FDE41227CE8F288E278D26D9
:101CF5008C25A91A7A007BFEC0030B8B2C752D222F
:101D0500752E9C8F328E318D308C2FD003122D6124
:101D1500EF251AF51A1218D31218C6121983751A57
:101D2500007849E2FC08E2FDEC1227CE8F288E27C9
:101D35008D268C25A91A7A007BFEC0030B8B2C758A
:101D45002D22752E9C8F328E318D308C2FD0031223
:101D55002D61EF251AF51A1218D31218C612198318
:101D6500751A00784BE2FC08E2FDE41227CE8F28B5
:101D75008E278D268C25A91A7A007BFEC0030B8B36
:101D85002C752D22752E9C8F328E318D308C2FD057
:101D950003122D61EF251AF51A1218D31218C6125F
:101DA5001983751A00784DE2FC08E2FDEC1227CE86
:101DB5008F288E278D268C25A91A7A007BFEC003D5
:101DC5000B8B2C752D22752E9C8F328E318D308C80
:101DD5002FD003122D61EF251AF51A1218D31218F8
:101DE500C6121983751A00A91A7A007BFEC0030B67
:101DF5008B2C752D22752E9C753200753100753032
:101E0500C8752F41D003122D61EF251AF51A121846
:101E1500D31218C6121983751A00A91A7A007BFE07
:101E2500C0030B8B2C752D22752ECD752F30D0034D
:101E3500122D61EF251AF51A1218D31218C61219A8
:101E450083751A00A91A7A007BFEC0030B8B2C75CB
:101E55002D22752E9C783BE2FC08E2FD08E2FE0887
:101E6500E2F5328E318D308C2FD003122D61EF25A6
:101E75001AF51A1218D31218C6121983751A00A961
:101E85001A7A007BFEC0030B8B2C752D22752E9CB8
:101E95007843E2FC08E2FD08E2FE08E2F5328E3105
:101EA5008D308C2FD003122D61EF251AF51A1218DB
:101EB500D31218C6121983751A00A91A7A007BFE67
:101EC500C0030B8B2C752D22752E9C753200753138
:101ED50000753080752F3FD003122D61EF251AF55F
:101EE5001A1218D31218C6121983751A00A91A7A6C
:101EF500007BFEC0030B8B2C752D22752E9C753235
:101F050000753100753000752F00D003122D61EF7B
:101F1500251AF51A1218D31218C6121983751A0044
:101F2500A91A7A007BFEC0030B8B2C752D22752E0A
:101F35009C7857E2FC08E2FD08E2FE08E2F5328EE5
:101F4500318D308C2FD003122D61EF251AF51A1221
:101F550018D31218C6121983751A00A91A7A007BAC
:101F6500FEC0030B8B2C752D22752E9C785BE2FC35
:101F750008E2FD08E2FE08E2F5328E318D308C2F45
:101F8500D003122D61EF251AF51A1218D31218C6AF
:031F95001219839B
:011F98002226
:101F9900C2AF751A00782EE2B40C00400302224346
:101FA900901FB0F8282873021FD402200602203897
:101FB90002206A02209C0220D502210E022147023A
:101FC90021800221B20221E3022214A91A7A007B9C
:101FD900FEC0030B8B2C752D22752ED0784FE2FC99
:101FE90008E2FD08E2FE08E2F5328E318D308C2FD1
:101FF900D003122D61EF251AF51A022243A91A7A84
:10200900007BFEC0030B8B2C752D22752ED77853C0
:10201900E2FC08E2FD08E2FE08E2F5328E318D307D
:102029008C2FD003122D61EF251AF51A022243A92C
:102039001A7A007BFEC0030B8B2C752D22752EDEC0
:102049007837E2FC08E2FD08E2FE08E2F5328E315B
:102059008D308C2FD003122D61EF251AF51A02222B
:1020690043A91A7A007BFEC0030B8B2C752D2275B0
:102079002EE5783FE2FC08E2FD08E2FE08E2F532CF
:102089008E318D308C2FD003122D61EF251AF51A60
:102099000222437847E2FC08E2FDE41227CE8F27AB
:1020A9008E268D258C24A91A7A007BFEC0030B8B02
:1020B9002C752D22752EEC8F328E318D308C2FD0D0
:1020C90003122D61EF251AF51A0222437849E2FC21
:1020D90008E2FDEC1227CE8F278E268D258C24A9A8
:1020E9001A7A007BFEC0030B8B2C752D22752EF3FB
:1020F9008F328E318D308C2FD003122D61EF251A3E
:10210900F51A022243784BE2FC08E2FDE41227CEDD
:102119008F278E268D258C24A91A7A007BFEC00371
:102129000B8B2C752D22752EFA8F328E318D308CBA
:102139002FD003122D61EF251AF51A022243784D8B
:10214900E2FC08E2FDEC1227CE8F278E268D258C26
:1021590024A91A7A007BFEC0030B8B2C752D2375DD
:102169002E018F328E318D308C2FD003122D61EFDD
:10217900251AF51A022243A91A7A007BFEC0030B1D
:102189008B2C752D23752E08783BE2FC08E2FD089F
:10219900E2FE08E2F5328E318D308C2FD003122DFC
:1021A90061EF251AF51A022243A91A7A007BFEC0AB
:1021B900030B8B2C752D23752E0F7843E2FC08E257
:1021C900FD08E2FE08E2F5328E318D308C2FD00306
:1021D900122D61EF251AF51A8060A91A7A007BFE83
:1021E900C0030B8B2C752D23752E167857E2FC082E
:1021F900E2FD08E2FE08E2F5328E318D308C2FD0F7
:1022090003122D61EF251AF51A802FA91A7A007B7E
:10221900FEC0030B8B2C752D23752E1D785BE2FCFC
:1022290008E2FD08E2FE08E2F5328E318D308C2F8E
:10223900D003122D61EF251AF51A1218D31218C6F8
:10224900C205D2AF782EE204F2C3940C4002E4F244
:012259002262
:10225A00C2AF751A00A91A7A007BFEC0030B8B2C39
:10226A00752D22752E8E1B8B2F753000753160D01F
:10227A0003122D61EF251AF51A1218D31218C6C2C5
:04228A0005D2AF22A8
:10232400C2B40000000000D2B50000000000D2B426
:10233400000000000022C2B40000000000D2B5007A
:1023440000000000D2B4000000000022D2B5D2B4D4
:102354000000000000C2B40000000000227F08C298
:10236400B500000000003312237ADFFAD300000026
:10237400000012237A2292B40000000000B2B500DB
:1023840000000000A2B40000000000B2B50000008C
:10239400000022122350E52D54FE12236150061230
:1023A400233A022397E52E122361E52F12236112AB
:1023B400233A22122350E52D54FE122361500612B3
:1023C400233A0223B7E52E122361500612233A0260
:1023D40023B7122350E52D4401122361227F0812F2
:1023E400237C33DFFAC3000000000012237A0000CC
:1023F400000000D2B4FF227F0812237C33DFFAD31B
:0D240400000000000012237A12233AFF228C
:10241100E528F82529F9AA29AC2ABC00030224429F
:10242100BA000302246CE67B08339291000000009D
:10243100D293000000000000C293DBED081C1A805B
:10244100D9BA000302246CE7FDE67B0833929100C0
:10245100000000D293CD339291000000000000C231
:102461009300CDDBE708091C1A80D6C2927819D8EF
:10247100FED2927819D8FEE52DAA2E2A14F8D29010
:10248100BA00030224A17B08A29033D2930000007A
:1024910000C293000000000000DBEDF6181A80E096
:0124A1002218
:030000000224A235
:0F24A200787FE4F6D8FD75A0007581BB02032397
:1024B100022873E86480F8E933E83360110460F0BE
:1024C100ED33EC337009E8FCE9FDEAFEEBFF220491
:1024D10060DED3EB9FEA9EE99DE8C2E78CF0C2F78C
:1024E10095F0400CE8CCF8E9CDF9EACEFAEBCFFB58
:1024F10012283E85D0F05804700320D5B3E804704B
:10250100075002B2D502287D92D5EC0460F7E4CCE5
:10251100C0E0C398F8603B94186008400DD0E0FB20
:10252100022855E4FBFAC9FC8028E830E406E4C936
:10253100FBE4CAFCE830E305E4C9CACBFCE8540774
:102541006010F8C3E913F9EA13FAEB13FBEC13FC7F
:10255100D8F130F52FC3E49CFCEF9BFFEE9AFEED22
:1025610099FDD0E0FBEF4E4D4C701222DB030228A7
:102571007AEC2CFCEF33FFEE33FEED33FDED30E76B
:10258100EB022855EF2BFFEE3AFEED39FDD0E0FBD3
:1025910050130BBB000302287DED13FDEE13FEEF7C
:0825A10013FFEC13FC022855A6
:1025A900EC4D6011E8497017ED33EC3304600DE42C
:1025B900FCFFFEFD22E933E8330470F802287312A8
:1025C900283E58046009E4CC2481500628500902A9
:1025D900287D28400302287AC0E0EB4A7044B9807C
:1025E90006D0E0FB022869EF4E701CBD8008EBFFA6
:1025F900EAFEE9FD80EBE98DF0A4FEE5F002269202
:10260900E9CDF9EAFEEBFFEF89F0A4FCE5F0CE890C
:10261900F0A42EFFE435F0CD89F0A42DFEE435F0C9
:102629008067EF4E7005BD80D780C3EF8BF0A4ACF7
:10263900F0EE8BF0A42CFCE435F0F8EF8AF0A42C32
:10264900E5F038FCE433CB8DF0A42CFCE5F03BF845
:10265900EE8AF0A42CFCE5F038F8E433CF89F0A435
:102669002CFCE5F038CF3400CE89F0A42FFFE5F03B
:102679003EFEE433C98DF0A42EFEE5F039CD8AF093
:10268900A42FFFE5F03EFEE43DFD33D0E0FB50070B
:102699000BBB000F02287DEC2CFCEF33FFEE33FE61
:0626A900ED33FD0228558F
:1026AF0002287DEC5D046005E8590470030228736D
:1026BF0012283E580460F6EC4860F2EC7004FDFE00
:1026CF00FF22C82481C85007C398500602287A9861
:1026DF0050CEF582E9294B4A7005AB820228697505
:1026EF00F0007C1A7880C3EF9BEE9AED99400DC3F2
:1026FF00EF9BFFEE9AFEED99FDE842F0DC23ACF084
:10270F00D0E0FFD0E0FED0E0FDAB8220E7101BEB66
:10271F0060BAEC2CFCEF33FFEE33FEED33FD0228F5
:10272F0055E803F830E705C0F075F000EF2FFFEE26
:0C273F0033FEED33FD40B830E7C280AA45
:10274B0074F8CC6480CCC86480C8F582046043C341
:10275B00EB9FF5F0EA9E42F0E99D42F0E89C45F0D4
:10276B0060305018E5825FFFE582F42B5582FB50F9
:10277B00210ABA001D09B90019088016E5825BFB16
:10278B00E582F42F5582FF50090EBE00050DBD00EA
:10279B00010CC3EB9FF5F0EA9E42F0E99D42F0E895
:0D27AB009C45F06007CC4820E701B3EC220C
:1027B800ED33EC33600A047003BD8004ECB2E7FC2F
:0127C80022EE
:1027C90075F020800E75F010800575F0087D007E8B
:1027D900007F003392D530D503122B11EC33401012
:1027E900EF33FFEE33FEED33FDEC33FCD5F0ED2294
:0E27F900E5F0247EA2D513CC92E7CDCEFF22D0
:10280700EDD2E7CD33EC3392D524814006E4FFFEC9
:10281700FDFC22FCE4CFCECDCC24E0501174FF8028
:10282700EDC3CC13CCCD13CDCE13CECF13CF0470C5
:07283700F030D5DE022B1189
:102D0500E540242CF8E60540227829301902782C74
:102D1500E475F001122BDF022A292012EB7F2ED257
:102D2500128018EF540F2490D43440D4FF30160B82
:102D3500EF24BFB41A0050032461FFE5416002157A
:102D4500410544E5447002054330190D7829E475C1
:102D5500F001122BDFEF022A9102365E7403D219BD
:102D65008003E4C219F5408B298A2A892BE4F541B1
:102D7500F543F544E54160077F20122D4080F5F5C8
:102D850042C213C212C214C215C217C218C21A1205
:102D95002D0EFF700D3019057F00122D51AF44AE79
:102DA5004322B42563C2D5C216122D0EFF24D0B41A
:102DB5000A00501E75F00A20D50DC541A42541F520
:102DC500417002D21580E0D212C542A42542F542D7
:102DD50080D524CFB41A00EF5004C2E5D2160230D4
:102DE50035D21380C2D21280BCD21480B8D2D5801D
:102DF500B6D21780B07F20122D402014077401B57C
:102E0500410040F1122D05FF122D40022D79D21AF5
:102E1500D2188091122D05FB122D05FA122D05F9F8
:102E25004A4B700679257A317BFF201433E54160E2
:102E35002FAF42BF00011F7E008E82758300122ACC
:102E45004260050EEE6F70F1C2D5EBC0E0EAC0E05E
:102E5500E9C0E0EE123090D0E0F9D0E0FAD0E0FB26
:102E6500122A29FF60A5EBC0E0EAC0E0E9C0E01244
:102E75002D40D0E02401F9D0E03400FAD0E0FBE5A4
:102E85004260DDD542DA8083D214809E12307560AF
:102E9500F7E542122887A942600BE542123118EF87
:102EA5007003D542F5EA30E702F404C3995077EA96
:102EB500F425420430E701E404F542800D12307533
:102EC50060C6EA05422542122887EA783FF630E7D0
:102ED50001E4254204D5420420170114123090E480
:102EE500C0E0123118783FE6601320E70714F612A8
:102EF5002D28802204F6D0E014C0E07F00122D2892
:102F0500E5426007122D1F1542800B301703122D65
:102F15001FD0E0022D79D0E00480C512307560A085
:102F2500E54204122887783FEAF6E54204201702B5
:102F3500600104240412309074FF04C0E0123118BB
:102F4500122D28E5422017026003122D1FD0E0B58F
:102F550042E87F45122D32783FE67F2B30E7047F2C
:102F65002DF404C0E0122D40D0E075F00A84C0F0C5
:032F7500122D29F1
:102F7800D0E0122D29022D79791080027908C21823
:102F8800C21A8008D2D5790A8004790AC2D5E4FA2F
:102F9800FDFEFF122D05FC7B08201313122D05FDE5
:102FA8007B1030120A122D05FE122D05FF7B20EC36
:102FB8003382D592D55013C3E43012069FFFE49EA6
:102FC800FEE42013039DFDE49CFCE4CBF8C213EC63
:102FD800700CCFCECDCCE824F8F870F38017C3EF8F
:102FE80033FFEE33FEED33FDEC33FCEB33FB99405E
:102FF80002FB0FD8E9EB301305F8D0E0C448B21350
:10300800C0E00AEC4D4E4F78207B0070C2EAC0E069
:10301800123092D0F0D0E0201304C4C0E0C4B21340
:10302800C0F0122D29D0F0D5F0EB022D79122BFF2C
:103038002E19532F80582DEA4C2DE6422F844F2FFE
:103048008C442F8C492DFF432F92552EC2462F209A
:10305800452E91473148502DEE2D2DF22E2E152B51
:103068002DF6232E132031332A00002E0D101203C3
:10307800754206122D05FC122D05FD122D05FE12B6
:103088002D05FF78380228B6790AA2D52015143004
:103098001709B910020404B9080104A2D5201802BE
:1030A8005001042014669214B541005032C0E07FEC
:1030B800203015177F30A21472187217500D123075
:1030C800E7C214C218C2177F30800F301703E9C057
:1030D800E0122D40301703D0E0F9D0E0B541CE30F2
:1030E80017177F30B9100C122D407F583016077F04
:1030F800788003B90803122D403014057F2D022D66
:10310800407F20201AF87F2B2018F322921480CFBA
:103118007F00B4070050052438F8E6FF22286E75B2
:103128006C6C29002D50434958D213122D053013C9
:10313800F8C213784130D504D2127842F6022DAA8B
:10314800122D052403B405004001E490312C93129C
:0F3158002D31743A122D31D215754104022F809A
:10316700E53A30150104F823282428F82278253079
:1031770015027828E475F001122BDF022A2960EC8A
:10318700C53E7002153D14C53E201504FF02369654
:10319700782574FFF5F0022BEFFF0236ACE53B60B4
:1031A70006D53B037F0022053EE53E7002053D2024
:1031B70015030236857825122BD6122A29FF60AC13
:1031C7007825E475F001022BDF1231AEEFC0E01273
:1031D70031A0D0E040F380A6D2158002C2158B251E
:1031E7008A268927E4F53CF53AF53DF53E753B001F
:1031F700C214C212C213C216123174FF7005AF3C5B
:103207007E0022B42530123174FF24D0B40A005056
:103217000C75F00AC53BA4253BF53B80E924CFB4E8
:103227001A00EF5002C2E502343ED21380D8D21200
:1032370080D4D21680D0EF1231A050051231D08041
:10324700ACEFC0E01231AED0E06F60A1EF606E125C
:10325700318580AA7401C53B6002F53B1231AEEFA0
:10326700605B20160E123167E475F001122BDFEF59
:10327700122A91D53BE6201604053A053C80C01278
:1032870031A4EFC0E01231A0D0E05004123185E440
:10329700FF20160E123167E475F001122BDFEF12D3
:1032A7002A91EF70DA201604053A053C8091E53B38
:1032B7006002053B1231D01231A4EF70C6301504FD
:1032C700E4123185E53C60030232057EFF7FFF2271
:1032D700E53B6002053B1231D0D218D2171231A458
:1032E700EF30180260D7C0E0123185D0E0AC3FADB7
:1032F70040AE41AF421235478C3F8D408E418F42E1
:1033070050071231AEC21780D420161020170205BD
:103317003C123167122BD6053A122B460231F4EFD5
:103327001231857908803B1231D01231AEEF608DB2
:10333700BF301B1231AEEF6084BF78028003BF58E5
:10334700DE7910801D1231D01231AEEF60E0790ABC
:10335700EFB42D04D2148019B42B028014123185D6
:10336700790AE53B6002053BE9C0E01231D0D0E0C5
:10337700F9D217E4FCFDFEFFE9C0E0ECC0E0EDC0C8
:10338700E0EEC0E0EFC0E01231A4EFF8D0E0FFD0EC
:10339700E0FED0E0FDD0E0FCD0F0E8604DB4610085
:1033A7004007B47B005002C2E524D0503DFA24F612
:1033B700500724F95034240AFAEAB5F000502BCF0D
:1033C700A9F0A42FFF92D5E9C5F0CEA4A2D53EFE61
:1033D70092D5E9C5F0CDA4A2D53DFD92D5E9C5F0BA
:0F33E700CCA4A2D53CFCC217808EE8C0E0201613
:1033F6002A201708053C301403122B1112316712CC
:103406002BD6053A20120B20130DEE8FF0122AA3AD
:103416008009122B468004EF122A91D0E0123185E2
:103426000231F4201610123167122BD6053AE53D0B
:10343600853EF0122AA380E8122BFF32B55333489B
:103446005832354C323142323148332A4F334C44AC
:10345600325B43332E4933675532D74632D745322E
:0C346600D74732392A34294E0000323D8D
:0D347200ED33EC3360065004EC6480FC2266
:10347F008F388E378D368C357FFF7EFF7DFF7CFF3B
:10348F00AB38AA37A936A835C3122B35602C7F80ED
:10349F007E967D187C4BAB38AA37A936A8351227F4
:1034AF004B600250157F807E967D187CCBAB38AA7F
:1034BF0037A936A83512274B5009AF38AE37AD367E
:1034CF00AC3522AF38AE37AD36AC351228078F3C4E
:1034DF008E3B8D3A8C39EC1227C9C8ECC8C9EDC99F
:1034EF00CAEECACBEFCBAF38AE37AD36AC35122400
:1034FF00B47B007A007900780012274B601A4018CD
:10350F00E53C24FFF53CE53B34FFF53BE53A34FF62
:10351F00F53AE53934FFF539AF3CAE3BAD3AAC394E
:05352F00EC1227C92287
:10283E00E9D2E7C933E833F892D5EDD2E7CD33ECE0
:07284E0033FC5002B2D52259
:10285500EC30E7100FBF000C0EBE00080DBD0004E4
:102865000BEB6014A2D5EB13FCED92E7FD2274FF90
:10287500FCFDFEFF22E480F8A2D574FF13FC7D80E9
:0228850080F0E1
:10288700F920E72824F950037907E4F42402FB1818
:10289700DBFDE624FB5014E9600DE4F618E604F6C8
:0F28A700B40A08E4F6D9F57401F60A22C2D52264
:1028B600ED33EC3392D5FA602AB4FF33EDC2E77BF1
:1028C600FF60067A2879DBE4227A2879E420D504A9
:1028D6007A2879DF224E614E002B494E46002D495B
:1028E6004E4600E47A08F608DAFC7B00740722E814
:1028F600C0E0ECC0E0EDC0E0EEC0E0EFC0E0EA759D
:10290600F010A4CAABF075F04DA42BFBE435F0FC37
:10291600EA2410FAEB34C5FBEC34D9FCEDC2E7FF30
:1029260075F056A4F42411C5F0F434C58FF0A42A2A
:10293600E5F03BE43CF620E7141229E9D0E0FFD0AD
:10294600E0FED0E0FDD0E0FC1226B28014F40412C2
:1029560029E9D0E0FFD0E0FED0E0FDD0E0FC122572
:10296600A9D0E0F8E6FAEDD2E7CD33EC332482FBCA
:10297600E4C3CF33CFCE33CECD33CD33DBF37B07BA
:1029860075F00A846004F6081B0AE5F0F6088FF075
:10299600740AA4FFACF08EF0740AA42CFEACF050BE
:1029A600010C8DF0740AA42CFDE435F0F608DBDE8C
:0329B60074072281
:10353400C219C21AC21BC21CF9E4F543F544FCFDCE
:10354400FEFFE91018EA201B0CB42D04D21BD32271
:10355400B42B02D32224D0504794095041240A307A
:103564001C15F88544F0740AA42872E74051C5F08C
:10357400704D85F044D322D21AC0E0E4FBFA7920DE
:1035840078411225A9ECF8EDF9EEFAEFFBD0E0FC56
:10359400E41227D31224B83019B41543D322240AD1
:1035A400201C20B4FE0720191AD219D32224EB6060
:1035B4000424E0700EA21B9219D21CC21BD322C396
:1035C400022873E4301C0BE544301B02F404A219F6
:1035D400921B301AEA254320D2E5A2E7921C50023E
:1035E400F404B4260050D8CCC0E0EDC0E0EEC0E056
:1035F400EFC0E0EC1229E9D0E0FFD0E0FED0E0FD1E
:10360400D0E0FC201C051225A980031226B2301B31
:06361400031227B8C322D7
:1029B9003F8000004120000042C80000447A000026
:1029C900461C400047C35000497424004B189680A8
:1029D9004CBEBC205A0E1BCA6753C21C749DC5AE9F
:1029E900FB60065407601C2323122A17EB54386036
:1029F90009122A03122A121225A9ECF8EDF9EEFAA6
:102A0900EFCB22EB122A1280F1543803241C9029AF
:102A1900B9FE93FC0EEE93FD0EEE930ECE93FF22BC
:102A2900BB010689828A83E0225002E722BBFE02AB
:092A3900E32289828A83E49322DE
:102A4200BB010CE58229F582E5833AF583E0225049
:102A520006E92582F8E622BBFE06E92582F8E22293
:0D2A6200E58229F582E5833AF583E49322AD
:102A6F00BB010989828A83F8E028F022500327F7F7
:102A7F0022BBFE05F8E328F3228A838982F8E493C8
:022A8F002822FB
:102A9100BB010689828A83F0225002F722BBFE0124
:022AA100F3221E
:102AA300BB010A89828A83F0E5F0A3F0225006F77E
:0F2AB30009A7F01922BBFE06F3E5F009F319227B
:102AC200E88FF0A4CC8BF0A42CFCE98EF0A42CFCB3
:102AD2008AF0EDA42CFCEA8EF0A4CDA8F08BF0A431
:102AE2002DCC3825F0FDE98FF0A42CCD35F0FCEB90
:102AF2008EF0A4FEA9F0EB8FF0A4CFC5F02ECD3955
:0F2B0200FEE43CFCEAA42DCE35F0FDE43CFC22C1
:10361A00C2D5E830E70FB2D5E4C39BFBE49AFAE4DB
:10362A0099F9E498F8EC30E717B2D5123650122C13
:10363A0067E4C39BFBE49AFAE499F9E498F88003F7
:10364A00122C6730D50DE4C39FFFE49EFEE49DFD76
:04365A00E49CFC22CE
:0E2B1100C3E49FFFE49EFEE49DFDE49CFC22D5
:102B1F00EB9FF5F0EA9E42F0E99D42F0EC6480C82D
:062B2F0064809845F022CD
:102B3500EB9FF5F0EA9E42F0E99D42F0E89C45F0F6
:012B4500226D
:102B4600BB010789828A83022CF95005E9F8022B1A
:0A2B560099BBFE05E9F8022BA52249
:0C2B6000E6FC08E6FD08E6FE08E6FF22A1
:102B6C00E493FCA3E493FDA3E493FEA3E493FF227C
:0D2B7C00E6FB08E6F908E6FA08E6CBF822C9
:102B8900E493F8A3E493F9A3E493FAA3E493FB226F
:0C2B9900ECF608EDF608EEF608EFF62268
:0C2BA500ECF208EDF208EEF208EFF2226C
:102BB100D083D082E493F208740193F208740293F3
:092BC100F208740393F27404732A
:0C2BCA00A42582F582E5F03583F5832216
:092BD600E6FB08E6FA08E6F92224
:102BDF00FAE6FB0808E6F925F0F618E6CA3AF622F7
:102BEF00FAE6FB0808E625F0F9F618E63AFAF622B7
:102BFF00D083D082F8E4937012740193700DA3A365
:102C0F0093F8740193F5828883E473740293686078
:062C1F00EFA3A3A380DF78
:062C25008A838982E4733A
:10365E00EFB40A07740D123669740A309811A899DE
:10366E00B8130CC2983098FDA899C298B811F630CC
:07367E0099FDC299F59922A4
:1036850010100B1236D8BF0D027F0A02365EAF1B33
:013695002212
:053696008F1BD2102281
:10369B00EFC394304009EFC3943A5003D38001C376
:0136AB0022FC
:1036AC00EFC394094006EFC3940E4003BF2003D32D
:0436BC008001C322A4
:1036C000CEEFCEEEC39461400BEEC3947B5005EE7B
:0836D00024E0FF22CFEECF221F
:102C2B0075F008758200EF2FFFEE33FECD33CDCC60
:102C3B0033CCC58233C5829BED9AEC99E5829840E3
:102C4B000CF582EE9BFEED9AFDEC99FC0FD5F0D6C0
:102C5B00E4CEFBE4CDFAE4CCF9A88222B800C1B9EA
:102C6B000059BA002DEC8BF084CFCECDFCE5F0CB28
:102C7B00F97818EF2FFFEE33FEED33FDEC33FCEB61
:102C8B0033FB10D703994004EB99FB0FD8E5E4F91C
:102C9B00FA227818EF2FFFEE33FEED33FDEC33FC09
:102CAB00C933C910D7059BE99A4007EC9BFCE99AFD
:102CBB00F90FD8E0E4C9FAE4CCFB2275F010EF2F42
:102CCB00FFEE33FEED33FDCC33CCC833C810D70742
:102CDB009BEC9AE899400AED9BFDEC9AFCE899F87D
:0E2CEB000FD5F0DAE4CDFBE4CCFAE4C8F92210
:0C2CF900ECF0A3EDF0A3EEF0A3EFF0224E
:0A36D8003098FDAF99C2987E0022E1
:00000001FF
